:020000040000FA
:1000000000308A002B2800001330840000080319F8
:10001000172801308D008C018C0B0C288D0B0B28C0
:100020004A308C008C0B12281528800B09280034CC
:1000300012309402031C2A2814308400FC308005FE
:100040000310800C800C000803192A2828280000BF
:10005000800B27287E2884011F3083058316861491
:100060008312861C6E2892011208643C031C5028DF
:1000700083160610831206148316051183120515C4
:100080000130930004208316061083120610831695
:10009000051183120511143093000420920A3428AC
:1000A00092011208643C031C6D288316061083120B
:1000B00006148316051183120515023093000420DF
:1000C000831606108312061083160511831205117C
:1000D000143093000420920A51282E28831606100B
:1000E000831206148316051183120515013093003F
:1000F000042002309300F73094001828930B7B28DB
:10010000831606108312061083160511831205113B
:0A0110001430930004202E28630031
:02400E00F93F78
:00000001FF
